:020000040000FA
:1000000001288B138C018316811700308600831220
:100010008611FF309200920B0B2883161030860059
:100020008312061A15288C0A1128831600308600C0
:100030008312861100308900831608148312080881
:100040008D000D18612864288E01831610308600FB
:100050008312061A2D288E0A29288316003086005E
:100060008312861103010C080E029100031D39282A
:1000700024289103031D3D2824289103031D4128B2
:1000800024289103031D452824289103031D492892
:1000900024289103031D4D2824289103031D512872
:1000A00024289103031D5528242883120030890039
:1000B00083160814831208088D008D0A0D18612814
:1000C00064280430860067280230860067280030E4
:1000D00089000D0888008316081555308900AA305C
:1000E000890088187128881450309400940B79285E
:1000F0008428FF3093008615930B7C28FF309300F3
:100100008611930B81287628940B842882309400E2
:10011000940B8B289F28FF3093008615930B8E2815
:10012000FF3093008611930B93288828FF309300AB
:10013000FF309300930B9A28930B9C289F28242828
:10014000FF309400940BA528B0289B3093008615AF
:10015000930BA8289B3093008611930BAD28A228FF
:0601600001308C0224288E
:02400E000900A7
:024200000000BC
:00000001FF
